:020000040000FA
:04000000000044298F
:080008008B138C1C2E288C10B8
:10001000BE0A00308A003E080739820716283A28AF
:100020003E28422846284A284E286928581C23285A
:10003000051550088E0051088F000C1010148316FF
:100040000C1483124229851552088E0053088F0024
:100050000C10101483160C14831242290C1C422914
:100060000C101010581C3728051158104229851102
:1000700058144229DF30E00059085128EF30E000E1
:100080005A085128F730E0005B085128FB30E000A7
:100090005C085128FD30E0005D085128FE30E0008A
:1000A0005E080F3954202929EF0000308A006F08BC
:1000B0008207403479342434303419341234023411
:1000C0007834003410347F34063406340634063471
:1000D00006346A187A28050803396802031D742853
:1000E000EC0B2629EA1426296A140330EB000F30A2
:1000F000EC002629EB0B262900308A00050803397D
:10010000E900E80D680D0C3969070F398207972857
:100110000C299C2897289C28972897280C290C297B
:10012000972897289C2897289C280C2997286A109C
:1001300005080339E800262905080339E800EA1C08
:10014000A3280130A4280830EA01D407031CA928F9
:10015000D50A683054020318B028EF000230B228E4
:10016000EF0001305502031CB828D5006F08D400F9
:100170005508031DC728B43054020318C728550872
:10018000D700B4305407D6000318D70ACF28550833
:10019000D700B4305402D600031CD703CF28DA01AD
:1001A000DB015408F0005508F10064307002031CB4
:1001B000DC28F000DB0AD528F1080319E428F10354
:1001C0006430F002DB0AD5280A307002031CEB28E9
:1001D000F000DA0AE4287008D900DD01DE015608D3
:1001E000F0005708F10064307002031CFA28F00098
:1001F000DE0AF328F10803190229F1036430F00242
:10020000DE0AF3280A307002031C0929F000DD0A17
:1002100002297008DC00262905080339E800EA1CD9
:100220001329013014290830EA01D4020318B82830
:100230000130D5020318B8286830D40703182329E1
:100240000130D507B8280230D507B828BF30E00004
:100250005F08E20006138617332106176008E200E4
:100260003321861342290830E3000612E21F3A299F
:1002700086163D298612000000000616E20DE30BEB
:10028000352909008B170900F130D300D100F03077
:10029000D200D000B430D600D701D401D501073048
:1002A000DF000030D9000030DA000030DB00003021
:1002B000DC000830DD000130DE004130C0000030DD
:1002C000BD00C100C200C300C400C500C600C70015
:1002D000C800BE01E6012030B8008312B901380819
:1002E00084003908840783169B001C141A088312A3
:1002F0008000B90A0F303902031D6F295A30B2004D
:10030000B300B4003930B500B6003230B000B101EE
:100310002A30B800B901BA01BB01BD0107309F0006
:1003200083160F308600F3308500831283169630D3
:10033000920083120F30920083164D3099002030C6
:1003400098008312903098008B170B1783168C142B
:1003500083128B178C1AAF29E61B002BAA298B134B
:100360001A08BC008C123B18152ABA1BDE2930086B
:1003700084003108840700083C02031DC929B10A22
:1003800005303102031DCA29B101B901FF30BA009D
:10039000A929B101380884003908840700083C0203
:1003A000031DDC29B90A05303902031DA929B10151
:1003B000B901FF30BA00A929B901A9293C08BA003E
:1003C000FF30BB0002308A003A080F390022CD000E
:1003D0004D080319262ABD0101303A02031DA9293F
:0803E0002808EE006D14A929A4
:10040000EF0002308A006F0882070034043404349D
:10041000063401340034003400340034053401342F
:10042000083400340034003400346D1C1D2A6E087A
:1004300003191C2AEE03A929ED01400884003D0898
:1004400084073C088000BD0ACD0BA929BD01BB0172
:1004500002308A003A080F39820744293D2A3D2A92
:100460008F2A9D2ABA2A44294429C02AD22AC82A76
:10047000A22A442944294429442921084202031C70
:100480004A2A031D5B2A20084102031C4A2A031D35
:100490005B2A562A42082302031C562A031D602A9F
:1004A00041082202031C562A031D602A4108D0007D
:1004B0004208D100642A2008D0002108D100642A13
:1004C0002208D0002308D10025084402031C712A09
:1004D000031D832A24084302031C712A031D832A57
:1004E0007D2A44082702031C7D2A031D892A43080C
:1004F0002602031C7D2A031D892A4308D2004408D2
:10050000D300BA01A9292408D2002508D300BA01D2
:10051000A9292608D2002708D300BA01A929410831
:10052000D9004208DA004308DB004408DC00450833
:10053000DD004608DE00BA01A9294108DF00DF0915
:10054000BA01A9294108A0004208A1004308A2005D
:100550004408A3004508A4004608A5004708A600D3
:100560004808A7000030E5002030E4000830E30030
:10057000BA01E32A540899008030E600BA01A9299B
:100580000830E5001130E7008130E600BA01A92902
:100590004108A8000830E5002830E4000130E300FD
:1005A000BA01E32A4108A9004208AA004308AB00A7
:1005B0004408AC004508AD000930E5002830E400EF
:1005C0000530E300BA0164088400000883169A002D
:1005D0008312650883169B009C111C1555309D00E5
:1005E000AA309D009C141C1183128C1FF52A8C13B9
:1005F000E50AE40AE30BE32AB901BA01BB01A92920
:100600008B130C1EA929661C112B650883169B00F1
:100610001C141A0883129900E50AE70BA929E601C0
:0A062000A92955089900E601A9294F
:02400E00613F10
:104200007400F5006C00EE007400F5006C00EE0028
:1042100000004300440049003900390020005300E9
:104220004500520056004F002000560031002E007D
:0242300030005C
:00000001FF
